:0800000000008A110A12072A10
:06000A00653083160313AC
:100010008600811281110115811401140230FF0044
:100020000030B421A421003049210030FF0000300D
:100030002B21063083120313A700A80106304921A3
:10004000FF3083120313A707031CA8032708280403
:10005000031D1E2804304921F52083120313A80034
:100060007F08A700FF3A031D392828083F3A0319E3
:10007000E520A42183120313861483120313A7011E
:10008000A8012030831203132802031D49280030E1
:10009000270203187C28831203132708FF0028086F
:1000A000D72183120313AA007F08A9000230492137
:1000B000831203132908FF002A082B21073083121B
:1000C00003132705A900AA012908073A031D702870
:1000D0002A08003A031D7028083049213D30CE21FE
:1000E000063049210230831203138606831203135C
:1000F000A70A0319A80A4128A42183120313A70100
:10010000A8012030831203132802031D8928003020
:1001100027020318B028831203132708FF002808BA
:10012000D72183120313AA007F08A90004304921B4
:10013000F52083120313AB007F082906031DA328B3
:100140002B082A06031DD5200630492102308312D0
:100150000313860683120313A70A0319A80A81282A
:10016000A421003049210030FF0000302B2107304E
:1001700083120313A700A80106304921FF30831220
:100180000313A707031CA80327082804031DBC2882
:10019000023049213A30FF003F302B2108304921FD
:1001A000831203138614D3280800831203138614C2
:1001B0006430FF000030B4218312031386100A302C
:1001C000FF000030B421D5280800831203138614E1
:1001D0000A30FF000030B42183120313861064300C
:1001E000FF000030B421E5280800831603138617AA
:1001F000013060210830602183120313B8000730FA
:10020000602183120313B9000310390C8312031306
:10021000A1003F30210583120313B9008316031395
:100220008601FA30CE218312031339088312031397
:10023000A200A100A001A3018312031338088312B6
:100240000313A100A0012108A3040030A204230885
:10025000FF002208080083120313A1007F08A000FA
:10026000A400A200A3010130FF0000308321083068
:10027000FF00831203132408832183120313A301B5
:100280000730FF002108A200A0008321FA30CE2110
:10029000080083120313A100F030831203138605B4
:1002A0000630FF00831203132108832183120313F6
:1002B0008617000000000000000000000000080099
:1002C00083120313A400A501A601831203132408BB
:1002D000260203187F290310A50C83120313861529
:1002E000F0308605861B782983120313A5137B291A
:1002F00083120313A51783120313A60A6529831219
:1003000003132508080083120313A0007F08A2002E
:10031000A30183120313220823020318A329201820
:1003200095298312031386139829831203138617C2
:10033000831203138615F03086050310831203130E
:10034000A00CA30A89290800103083120313860029
:100350000230FF000030B421831203138601023003
:10036000FF000030B421080083120313A1007F08AE
:10037000A000A201A3018312031321082302031D7D
:10038000C329200822020318CD293D30CE21831233
:100390000313A20A0319A30ABB290800831203133B
:1003A00081000B11831203130B1DD2290800831245
:1003B0000313A200A1007F08A000A301220883125A
:1003C00003178F0083120313A10120088312031760
:1003D0008D00831603178C170C140C140C14831245
:1003E00003170E0883120313A300A000A101A201AA
:1003F000831203170C0883120313A000A101200825
:10040000A2040030A3042208FF0023080800CF3014
:10041000FE000230FF0080308A110A12AE228A11DB
:100420000A1283120313AD007F08AC00D130AE0076
:100430000230AF00831203132C08B0002D08B10066
:10044000FF30AC07031CAD03300831040319972AB1
:1004500004302E07B000B101B10D2F08B1073008EC
:10046000FE003108FF0080308A110A12AE228A1184
:100470000A1283120313B3007F08B2002E08FE0095
:100480002F08FF0080308A110A12AE228A110A1248
:1004900083120313B500B1007F08B400B00002302E
:1004A0002E07B000B101B10D2F08B1073008FE00D2
:1004B0003108FF0080308A110A12AE228A110A1216
:1004C00083120313B100B7007F08B000B600831297
:1004D00003133208B6003308B700FF30B207031C1D
:1004E000B303360837040319902A3408FE00350890
:1004F000FF0080308A110A129B228A110A1283128D
:100500000313B600300884008313311883173608AC
:100510008000B40A0319B50AB00A0319B10A672AA0
:10052000063083120313AE070318AF0A1A2A8A1182
:100530000A1205280800003A0319A22A803A031972
:10054000A92A00347E08840083137F1883170008CB
:1005500008007F088A007E0882000800003A03191C
:10056000B62A803A0319C02AFF0100347E088400AD
:1005700083137F1883170008FF00840A000808000F
:100580008A110A12A922FD00FE0FFF03FF0A8A1139
:100590000A12A922FC007D08FF007C080800013433
:1005A0000034D73402343A34003401340034003497
:00000001FF
